:101C000012C02CC02BC02AC029C028C027C026C0A3
:101C100025C024C023C022C021C020C01FC01EC0B8
:101C20001DC01CC01BC011241FBECFE5D4E0DEBF09
:101C3000CDBF10E0A0E6B0E0E2EBFFE102C005900E
:101C40000D92A236B107D9F710E0A2E6B0E001C0CC
:101C50001D92A83EB107E1F767D0A9C1D1CFCF93BC
:101C6000DF93EC01A0916400B091650083E0FD0179
:101C700080935700E89507B600FCFDCF1092E7006F
:101C800071E014C0262F30E0FE01E20FF31F5181F6
:101C900040E0808190E0842B952BF9010C0170933A
:101CA0005700E89511246E5F6093E7006091E700AC
:101CB000603440F385E0FD0180935700E89507B656
:101CC00000FCFDCFDF91CF91089581E18093570013
:101CD000E895E0E0F0E0099508958CB95E9BFECFB1
:101CE0005E9A08955F9BFECF8CB10895FC0170E869
:101CF00080E090E0A1E2B0E1508140E084279527A8
:101D000068E09C01220F331F97FF02C02A273B2760
:101D10006150C901B1F7715011F03196EDCF309398
:101D2000E600209363000895AF92BF92CF92DF92B6
:101D3000EF92FF920F931F93CF93DF93F8942EE0CF
:101D400088E190E00FB6F894A89581BD0FBE21BD43
:101D50008AE196E09BBD8ABD1FBC8DE08EBD8F9A47
:101D60001BB888E18AB986E880BD10BC88E089B9D3
:101D7000109263001AE0A89508B604FE0DC088B75B
:101D8000806188BF809163008130C9F082B3805840
:101D900082BB115009F499DF5F9BEDCF8CB120918C
:101DA0006300E22FF0E0E05AFF4F9081891721F4A1
:101DB0002F5F20936300DFCF10926300DCCF14E12C
:101DC00003E408B604FE0DC088B7806188BF0CB973
:101DD0005E9BFECF5E9A82B3805882BB115009F49D
:101DE00074DFA8955F9BEDCF8CB1813051F71EBC9D
:101DF00010926200109265001092640010E0EE24D0
:101E000075E1D72EC0E8D0E066E0C62E51E1B52ED0
:101E1000AA24A394E3945F9BFECF9CB19093E60029
:101E20005F9BFECF8CB1809580936300E91609F02B
:101E30009CC0E81609F099C090916200292F2058A3
:101E40005F9BFECF8CB1E92FF0E0EA59FF4F808312
:101E50009F5F9217A9F7909362005F9BFECF0CB132
:101E60005F9BFECFFCB0892F90E08A5190403EDF0F
:101E70008091E600081709F074C080916300F8169D
:101E800009F06FC0809164009091650080509C4182
:101E9000B8F01BC0FE01E81BF109CF018A599F4F22
:101EA000DEDE8091640090916500805C9F4F90938E
:101EB000650080936400809162008054809362008A
:101EC00080916200882331F702C010926200409135
:101ED000640050916500FCE140305F07C0F5B092AE
:101EE0005700E895A09263001092E70020E0BA0145
:101EF0006058704014C0A22FB0E0CB018A0F9B1F26
:101F0000FC019491322F3F5FAA59BF4F8C919817D3
:101F100029F02093E7001092630005C0232F27FFCC
:101F2000EACF2093E70080916300882321F0CCB8AA
:101F30005E9BFECF0FC0DCB85E9BFECF5E9A1F5F3C
:101F400040585040509365004093640005C0CCB8A1
:101F50005E9BFECF5E9A10E0A89582B3805882BB4C
:101F600009C0DCB85E9BFECF03C0DCB85E9BFECF31
:101F70005E9A1F5F143030F45F9BFECF8CB18430CB
:101F800009F048CF86E08CB95E9BFECF5E9A1111B6
:101F9000FFCF9BDE80E090E0DF91CF911F910F910A
:101FA000FF90EF90DF90CF90BF90AF900895F8949E
:021FB000FFCF61
:021FB2006400C9
:0400000300001C00DD
:00000001FF
